:10000000BE01A828A70085100510051083168510CD
:10001000051005100F30860583122708BE182E28FC
:100020003A30A100983067203330A60042201330C8
:10003000A10088306720422064306620422064306E
:1000400066202230A600422028302D200C302D20A2
:1000500006302D20BE1427082E283E14A6003E1C74
:100060003C280510033C031C412841200730A10017
:10007000D0306720031408003E14FE3C0319A32867
:1000800005143E1C3E1085140F3086052608F039F5
:1000900086048510A60E3E184228323066200314CE
:1000A000080003178D0083168C130C1483120C08A0
:1000B000A328A301A200FF30A207031CA307031C6F
:1000C000A3280330A100DF3067205B28A101E83EB0
:1000D000A000A109FC30031C7028A00703186D289C
:1000E000A0076400A10F6D2820187628A01C7A288C
:1000F00000007A280800A2000530A8002308210289
:10010000031D84282208200204300318013003193B
:1001100002302805031DFF30A3281030A800A101DC
:10012000A001A70CA60C031C9B282208A0072308EB
:100130000318230FA107A10CA00CA50CA40CA80B5D
:1001400091282408A3288313031383126400080052
:10015000831607309F0081010F30860085018312CE
:10016000FE308A01022001308A01022020308A01FB
:10017000022020308A01022041308A0102204330CF
:100180008A01022054308A01022049308A0102206B
:1001900056308A01022041308A01022020308A0133
:1001A000022020308A01022052308A01022045308C
:1001B0008A0102204C308A01022045308A01022047
:1001C00020308A01022020308A010220FE308A017C
:1001D0000220C0308A01022020308A010220203013
:1001E0008A01022020308A0102205B308A0102202D
:1001F00039308A0102205D308A0102203D308A01B7
:1002000002204F308A0102204E308A0102202F3016
:100210008A0102204F308A01022046308A010220E2
:1002200046308A0102208A117A2164004E08003C7F
:100230008A110319132964005008393C8A110319E3
:1002400023298A01132964308A015920FE308A014A
:10025000022001308A01022020308A010220203051
:100260008A01022049308A0102204E308A01022090
:1002700047308A01022052308A01022045308A012B
:10028000022053308A01022045308A0102202030AA
:100290008A01022050308A01022041308A01022066
:1002A00053308A01022053308A01022020308A0113
:1002B000022020308A0102200130A300F4308A019C
:1002C0005A208A115D2264004C08003C8A110319EF
:1002D000B0288A11EB228A11042364004C08013CE7
:1002E0008A110319B028043085068316051183127C
:1002F0008A01B028CE01FF30D000703086000F3068
:100300000605B200B3013208A0003308A100A30122
:100310000E308A017B208A11031D94292A30D000D7
:100320000130CE008A11B4293208A0003308A100A0
:10033000A3010D308A017B208A11031DA5293030CD
:10034000D0000130CE008A11B4293208A000330851
:10035000A100A3010B308A017B208A11031DB4295F
:100360002330D0000130CE00B03086000F300605BB
:10037000B200B3013208A0003308A100A3010E307F
:100380008A017B208A11031DCB293130D000013036
:10039000CE008A11EB293208A0003308A100A30186
:1003A0000D308A017B208A11031DDC293230D000F8
:1003B0000130CE008A11EB293208A0003308A100D9
:1003C000A3010B308A017B208A11031DEB293330F6
:1003D000D0000130CE00D03086000F300605B200CC
:1003E000B3013208A0003308A100A3010E308A0136
:1003F0007B208A11031D022A3430D0000130CE0048
:100400008A11222A3208A0003308A100A3010D306E
:100410008A017B208A11031D132A3530D000013058
:10042000CE008A11222A3208A0003308A100A301BD
:100430000B308A017B208A11031D222A3630D0001E
:100440000130CE00E03086000F300605B200B30167
:100450003208A0003308A100A3010E308A017B20DE
:100460008A11031D392A3730D0000130CE008A119D
:10047000592A3208A0003308A100A3010D308A01D7
:100480007B208A11031D4A2A3830D0000130CE006B
:100490008A11592A3208A0003308A100A3010B30A9
:1004A0008A017B208A11031D592A3930D00001307E
:1004B000CE0032308A0159200800FE308A01022025
:1004C00001308A0102200130CD00CE018A017A215B
:1004D0000A308A01592064004E08003C8A11031931
:1004E000652A64308A015920640050082A3C8A1128
:1004F000031D7E2ACC0108008A11912A640050084D
:10050000233C8A11031D912A640005304D028A1193
:1005100003188E2A8A01652A8A11912A0130CC009B
:100520000800640005304D028A110318A42AFF3028
:100530004D07B200FF300318013EB3003208443EBD
:10054000840050088000CD0AFE308A01022001306C
:100550008A010220640002304D028A11031CBF2A66
:100560000230CF0064004F084D028A11031CBF2ADD
:100570002A308A010220CF0A8A11031DB22A6400A0
:100580004D08053C8A11031DE92AFE308A0102202C
:10059000C0308A01022020308A01022020308A01E6
:1005A000022020308A01022020308A0102202030DF
:1005B0008A01022020308A01022020308A01022094
:1005C0005B308A01022023308A0102205D308A01DB
:1005D00002208A01652ACF01640004304F028A118B
:1005E0000318032B4F088A015120B200B3014F08B2
:1005F000483E8400320880000A308A015920CF0A20
:100600008A11031DEC2A0800CF01640004304F0258
:100610008A110318312B4F08443E84000008B200B1
:10062000D0303207B200FF300318013EB3004F084C
:10063000443E8400320880004F08483E8400000891
:10064000B200D0303207B200FF300318013EB300D1
:100650004F08483E840032088000CF0A8A11031DEB
:10066000052B4408A600A701E830A2000330A30030
:100670008A018D20B2002508B3004508A600A70115
:100680006430A200A3018A018D20B4002508B500C2
:100690003208B40733080318013EB5074608A60020
:1006A000A7010A30A200A3018A018D20B600250807
:1006B000B7003408B60735080318013EB7074708E6
:1006C000B6070318B70A4808A600A701E830A20039
:1006D0000330A3008A018D20B8002508B90049081D
:1006E000A600A7016430A200A3018A018D20BA00F0
:1006F0002508BB003808BA0739080318013EBB07B4
:100700004A08A600A7010A30A200A3018A018D2091
:10071000BC002508BD003A08BC073B080318013E91
:10072000BD074B08BC070318BD0A3C083602CC00C5
:08073000080063008A01992B07
:02400E00753FFC
:084200003100320033003400EC
:00000001FF
